:10000000020FFDC299900139E0FF900138E06F6066
:0F0010000A1214E82408F8E6F59922C2072232F2
:0300230002126660
:03002B0002108937
:1000330002001EBB010689828A83F0225002F72246
:10004300BBFE01F322EF8DF0A4A8F0CF8CF0A4281F
:10005300CE8DF0A42EFE22BC000BBE0029EF8DF046
:1000630084FFADF022E4CCF875F008EF2FFFEE33F8
:10007300FEEC33FCEE9DEC984005FCEE9DFE0FD5A7
:10008300F0E9E4CEFD22EDF8F5F0EE8420D21CFE7B
:10009300ADF075F008EF2FFFED33FD4007985006E4
:1000A300D5F0F222C398FD0FD5F0EA22C2D5EC3089
:1000B300E709B2D5E4C39DFDE49CFCEE30E715B23D
:1000C300D5E4C39FFFE49EFE12005AC3E49DFDE402
:1000D3009CFC800312005A30D507C3E49FFFE49EC3
:1000E300FE22C5F0F8A3E028F0C5F0F8E5821582FA
:1000F30070021583E038F022E88FF0A4CC8BF0A4D3
:100103002CFCE98EF0A42CFC8AF0EDA42CFCEA8EE6
:10011300F0A4CDA8F08BF0A42DCC3825F0FDE98F09
:10012300F0A42CCD35F0FCEB8EF0A4FEA9F0EB8F00
:10013300F0A4CFC5F02ECD39FEE43CFCEAA42DCECD
:1001430035F0FDE43CFC2275F008758200EF2FFFCB
:10015300EE33FECD33CDCC33CCC58233C5829BED9C
:100163009AEC99E58298400CF582EE9BFEED9AFDA0
:10017300EC99FC0FD5F0D6E4CEFBE4CDFAE4CCF950
:10018300A88222B800C1B90059BA002DEC8BF084C3
:10019300CFCECDFCE5F0CBF97818EF2FFFEE33FE91
:1001A300ED33FDEC33FCEB33FB10D703994004EB49
:1001B30099FB0FD8E5E4F9FA227818EF2FFFEE3315
:1001C300FEED33FDEC33FCC933C910D7059BE99A27
:1001D3004007EC9BFCE99AF90FD8E0E4C9FAE4CCB8
:1001E300FB2275F010EF2FFFEE33FEED33FDCC3322
:1001F300CCC833C810D7079BEC9AE899400AED9B0B
:10020300FDEC9AFCE899F80FD5F0DAE4CDFBE4CCE9
:10021300FAE4C8F922EB9FF5F0EA9E42F0E99D4229
:10022300F0E89C45F022E8600FECC313FCED13FDEE
:10023300EE13FEEF13FFD8F122E493FC740193FD58
:10024300740293FE740393FF22A42582F582E5F0E2
:100253003583F58322E493FB740193FA740293F9D3
:1002630022EC8EF0A4CCC5F0CCCDF8EFA4CEC5F033
:100273002DFDE43CFCE8A42EC8C5F03DFDE43CFCA8
:10028300EFA4FFE5F028FEE43DFDE43CFC228F36BD
:100293008C378D38E4F544F545F542F543F539E5FA
:1002A30039C39536400302037B900099E0FF65391B
:1002B300701CE54E2FFFE4120876FCA3E0FD120844
:1002C30061FEA3E0C39DF541EE9CF54080641208F6
:1002D3004D12086D12093A8F3D8E3C8D3B8C3AE5E9
:1002E3004E2539FFE4120858120950AF3DAE3C12B7
:1002F30001868E3E8F3F12084D12086D12094595F7
:100303003FFFEE953EAB07FAE4F9F8AF3DAE3CADE7
:100313003BAC3A1201868E3E8F3F900099E0254E0A
:10032300FFE4120858FEA3E0C3953FF541EE953E66
:10033300F540C3E540648094805005E4F540F54101
:10034300D3E5419543E540954240148546478542B0
:10035300448543458539468540428541438014D3CE
:10036300E5419545E5409544400985394785404435
:1003730085414505390202A2E5432545FFE542359E
:1003830044FEC3EF9538EE953750057EFF7FFF227D
:10039300E537C313FEE53813FFC3E5439FF541E596
:1003A300429EF540FEAF417C007D0A1200481209CF
:1003B30023EDD3941F40027D1FEDAC37AD381208F7
:1003C300DFCEC313CE13D8F9F53F8E3E2543F54355
:1003D300E53E3542F542E53F2545F545E53E3544E5
:1003E300F544E545AE447807C333CE33CED8F9FFA1
:1003F3001209239000F6E07002A3E070051208FCD6
:10040300800D12092DCEC313CE13D8F91208B512DD
:10041300095ACEC313CE13D8F9FD9000B0E546F0C8
:1004230075F040A485F048F549E54612090C5002E1
:10043300AD07E54612088BC333CE33CED8F9120885
:100443009DAD07AC06E546700AE53614B54704C210
:1004530006801BE53614B54608E5477004D20680CE
:100463000DE546C395475004D2068002C206300606
:100473000CED2549F549EC3548F5488022E5494519
:10048300487011E53675F040A4AEF024FFF549EE4F
:1004930034FFF548C3E5499DF549E5489CF548AE69
:1004A30048AF4922C205754E06200307D2037F04D5
:1004B3001212AA7D0C7C007F04120291EFF47002E9
:1004C300EEF46002C2049000F5E0F960030205B1A6
:1004D3009000F4E06003020581EFF47002EEF46033
:1004E3000B7401F09000D704F0020601854E32121E
:1004F30009AD400302060112098EE532120982E0BA
:10050300FAA3E0FBD39DEA9CE5324007120990C3AE
:10051300EB8014120982E0FCA3E0FDE532120A220B
:10052300F583E0FAA3E0C39DF534EA9CF533D3E504
:10053300349408E5339400502174EA25321209A556
:10054300E0703612098EE532120982ECF0A3EDF069
:1005530012098EE532120A72800E12098EE53225D7
:10056300E02402F582E43400F583ECF0A3EDF074AB
:10057300EA25321209A57432F005320204F2EFF4CF
:100583007002EEF4600D9000D7E070729000F504F5
:10059300F0806BE49000F4F0854E321209AD505EAA
:1005A30074EA25321209A57432F0053280EDE9644C
:1005B30001704B9000F4E06011EFF47002EEF47000
:1005C3003DF09000D77402F08034EFF47002EEF443
:1005D30070269000D7E070269000F5F0A3F0A312E8
:1005E3000A2C854E321209AD501474EA25321209D1
:1005F300A57432F0053280ED9000F47401F09000A0
:10060300F5E064017061EFF47002EEF460089000AD
:10061300D4EEF0A3EFF09000F6E0FEA3E07802CE74
:10062300C313CE13D8F9F5359000B0E02430FF1290
:10063300121A7F2012121AE53575F064120681E54D
:100643003575F06484E5F075F00A120681E53575B9
:10065300F00A84E5F02430FF12121A7F0D12121AE9
:100663007F0A12121A8003120A2D9000D4E0F4704C
:1006730003A3E0F46004754D0222E4F54D228424C3
:1006830030FF12121A22E4F532F5F875FB3FD2015E
:1006930053D57F43D501E5F854F84407F5F853F8EB
:1006A300BF75F90F75FA329081037440F0E4F5E8F1
:1006B300F5C0908030F090FC00E04440F0E58654B3
:1006C300F04407F586E4F54B12143175A1A575D5F1
:1006D3008075D67FE532601F908030E0547FF0E074
:1006E30054FE4401F0C2AF438702000000E044809F
:1006F300F0E054FEF0D2AF9000D8E0FF120A1A40A7
:1007030003020814AEFBEE60CBEF600214F0E4FDCD
:10071300ED120A1140030207ED7E007401A80508DB
:100723008005C333CE33CED8F9FFACFBECFBEF5BD4
:1007330070030207E9A8057401088002C333D8FCDB
:10074300F5FBEDFF7E00700885E23385E1348044DC
:10075300EF64014E700885E43385E3348036EF643B
:10076300024E700885E63385E5348028EF64034E36
:10077300700885D93385E734801AEF64044E700816
:1007830085DB3385DA34800CEF64054E700685DD36
:100793003385DC34E532702CE53424FCFFE5333457
:1007A300FFFEE54B2DFC120A51EEF0A3EFF0E5340A
:1007B3002404FFE43533FEEC120A83F583EEF0A341
:1007C300EFF08022E54B2DFF120A51E0FAA3E0C3BC
:1007D3009534EA9533503AEF120A831209CCD39534
:1007E30034EE9533402B0D020713E54B2406120913
:1007F300EF50087406254BF54B800DE4F54BE532BD
:10080300700675320143F82012143175A1A5020652
:10081300D7E4F5F875FB3FE58654F0440DF58612F1
:100823000A44908030E04440F053D57F43D5017FA4
:10083300017E001214B975D580E4F5D6F54B12117B
:10084300CC120A7CC20175E8E322900099E0AD4E18
:100853007C002DFFEC33FEEF25E0FFEE33FE741634
:100863002FF58274003EF583E022FAA3E0FBED2529
:1008730039FFEC33FEEF25E0FFEE33FE749A2FF5DC
:100883008274003EF583E02290169293FCFFEDC341
:100893009FFFE49400FEEF780522FFECFDC3748014
:1008A3009DFDE49400FC0200AF75F0029000160277
:1008B300024CFFC3EB9FFFEA9E9000F6F0A3EFF01C
:1008C300EDFF9000F6E48FF00200E5E50090009A5A
:1008D30075F00212024CE0FEA3E0FF22FFC3742076
:1008E3009FFFE49400FE120048EF780622C3EB9FBB
:1008F300EE6480F8EA64809822ED75F004A4FF901A
:1009030000F6E5F0F0A3EFF02290169293FFEDC30B
:100913009F22E500C313FEE50013FFC3E5009F22FA
:10092300AC42AD4312005AAD07229000F6E0FAA3A1
:10093300E0FBAE02780222FEA3E0FFAD03AC0202AD
:100943000264FEA3E02BFFEE3AFEC3EF22FEA3E018
:10095300FBAA06E4F9F8229000F6E0FEA3E0780291
:1009630022AC00AD0012005AAD0722E53225E02487
:100973009AF582E43400F583E0FEA3E0FFE5322537
:10098300E02402F582E43400F58322E53225E024F5
:100993009AF582E43400F583E0FCA3E0FD2274EAD7
:1009A3002532F582E43400F58322E54E2404FDE488
:1009B30033FCC3E5329DEC6480F874809822E53201
:1009C30025E024B1F582E43400F583E0FEA3E022C0
:1009D30074D92532F582E43400F58322E53275F0CB
:1009E3000AA4242AF582E43400F58322FFE433C306
:1009F300FE7860E6FDEF9D7480F86E982225E02472
:100A030016F582E43400F583EEF0A3EFF022C394ED
:100A1300067480948022E0C3940574809480222518
:100A2300E0249AF582E4340022F074FF9000D4F0BD
:100A3300A3F022E53290169693FF7862E6FEEF5E0E
:100A43002275F90A75F8409081037457F02225E066
:100A530024FAF582E43400F583227860E62401FF6A
:100A6300E433FEC32225E024B1F582E434002225D9
:100A7300E02416F582E43400229000D37405F022BA
:100A830025E0240EF582E4340122E4F532E5321246
:100A93000A114003020B62120980E0FCA3E0FD127D
:100AA3000B738F33E532120990120B738F34EF649B
:100AB300026007EF64036002C204E5337030E5347B
:100AC300701B120A36700E1209A1E06003020B5D5F
:100AD300EF4EF680001209A17402F0807D120A36EF
:100AE30060691209A1E07072EFF45EF68015E534D7
:100AF300700C12096EEEF0A3EFF0E4FD80577862FC
:100B0300E66011E532120A72120979EEF0A3EFF0F2
:100B13007D028041120980E0FEA3E0FFE532120965
:100B2300907B1E7A0012145FEF60201209A1E0701F
:100B33002912096EEEF0A3EFF0E532120A22120930
:100B4300CCFFE532120A007D02800A12096EEEF034
:100B5300A3EFF0AD34AF321215120532020A9078CA
:100B630062E69000D6F06004754D0122E4F54D2253
:100B7300E5329016969378625624FF92057B1E7A8F
:100B830000AF3212111022E4F530F52FF52EF52DBA
:100B9300F53175E8E3FF7EC27D01FC120ED2908031
:100BA30030E04440F075A081E4F5A375A24B75A134
:100BB300A5D2AF120F719080077402F0C287121290
:100BC300EBE48F308E2FF52EF52DAD2EAC2D78085E
:100BD3001202298F1D85301E12116F9000D4E0FE82
:100BE300A3E0FFF47002EEF4601475310375530152
:100BF30074362FF58274153EF583E493F554900013
:100C0300D6E0603F75530175310324FE601924FE5D
:100C1300601A24FC601B24F8601C24F0601D241F50
:100C2300701E7554F4801C7554F580177554F38049
:100C3300127554F0800D7554F280087554F18003D9
:100C4300E4F553E5536091D3E51C941474809480C8
:100C53004086E4F51CF553F51CC2AFAF311213CD3A
:100C6300D2AF020BDB900098E07015C2009000D861
:100C7300F0F54B1211CC9000987402F0754A3222B1
:100C8300900098E064026003020D45200003020D0A
:100C930045C200154AE54A6003020D457861F6F541
:100CA30032120A5DE5329FEE1209BA4003020D418A
:100CB300E4FFEF120A1A501CE532120A681209996E
:100CC300E5321209E175F002EF12024CECF0A3EDEC
:100CD300F00F80DE74D925321209D7E4F0E53278BB
:100CE3006066605A1209C1FFE532120A001209C197
:100CF300FFE532120982EEF0A3EFF0E532120A119A
:100D0300502DE53225E025E02478F582E43416F50C
:100D130083E493FE740193FFE53225E024C7F58253
:100D2300E43400120A097D02AF32121512800A74EC
:100D3300EA25321209A57432F00532020CA4785563
:100D4300760122908109E054E06004E044E0F0E59C
:100D5300FB30E00975FB0185E22185E122E5FB30EB
:100D6300E10975FB0285E42385E324E5FB30E20911
:100D730075FB0485E62585E526E5FB30E30975FB70
:100D83000885D92785E728E5FB30E40975FB10853D
:100D9300DB2985DA2AE5FB30E50975FB2085DD2BA8
:100DA30085DC2CE4FFEF120A11502DEF25E02421FE
:100DB300F8E6FC08E6FDE54B2F120A68F583ECF034
:100DC300A3EDF0EFFDE54B2DFDE433FC7860E66D1C
:100DD3007001EC60030F80CDE54B2406FFE433D3B1
:100DE3001209F34007D200E4F54B80067406254B45
:100DF300F54B1211CC9000D8E0600214F09000F98A
:100E0300E0FF9000F8E0FE6F6006A3EEF075A1A589
:100E130022E4F532120A5DE5329FEE1209BA40036D
:100E2300020ED11209D3E004F01209D3120A1940B9
:100E3300051209D3E4F0C2ADE5321209C3FF12096A
:100E4300DFC083C0821209D3E0D082D08375F00261
:100E530012024CEEF0A3EFF0D2ADE4F533F534F526
:100E630035F53674FFF537F538E4FFEF120A1A50FB
:100E7300351209DF75F002EF12024CE0FCA3E0FD2E
:100E83002534F534EC3533F533D3ED9536EC953520
:100E930040048C358D36C3ED9538EC953750048C72
:100EA300378D380F80C5C3E5349536FFE533953567
:100EB300FEC3EF9538FFEE9537FE7C007D031200ED
:100EC3005AE532120A22120A090532020E17228F3C
:100ED300358E348D338C32E4900138F0A3F09001D9
:100EE30022F0A3F0C2079080197405F0908018F0E7
:100EF300E4F538C3E5389408748094805052121492
:100F0300F62436F582E43416F58312023CAB35AA97
:100F130034A933A832C312021870311214F62456BE
:100F2300F582E43416F583E493FE740193FFC3E47E
:100F33009FF537E49EF5361214F62458F582E4340F
:100F430016F5837401934480F5D88004053880A393
:100F5300E5386408601775C824E536FFF5CBAE376E
:100F63008ECA8FCD8ECCD2CE759850D2AC227860FB
:100F7300760AE4FFFEEEFD7C00C3940A748094803D
:100F8300502AC3ED120A12EE501125E025E0247613
:100F9300F582E43416F5837401800390168893FD7B
:100FA300AC070F74562CF8A6050E80C9908030E06C
:100FB3004440F075D580E4F5D6D2AD121402120A7E
:100FC30044D2ADC200E49000D6F07862F6F54D123B
:100FD3000A7CD202C201C203E49000F5F09000F44F
:100FE300120A2CE49000F6F0A3F07855F6900098DE
:100FF300F09000F9F09000F8F022787FE4F6D8FD45
:10100300758164021044020B8AE493A3F8E493A36A
:101013004003F68001F208DFF48029E493A3F85437
:1010230007240CC8C333C4540F4420C8834004F4BA
:1010330056800146F6DFE4800B01020408102040CD
:1010430080901525E47E019360BCA3FF543F30E5F7
:1010530009541FFEE493A360010ECF54C025E06042
:10106300A840B8E493A3FAE493A3F8E493A3C8C510
:1010730082C8CAC583CAF0A3C8C582C8CAC583CA01
:10108300DFE9DEE780BEC0E0C0F0C083C082C0D02D
:1010930075D000C000C001C002C003C004C005C0B9
:1010A30006C007E5D530E03F43D501300108900085
:1010B300D8E004F0803C121325E55245516008E561
:1010C30052155270021551051FC3E51F9480748099
:1010D30094804006751F001214FDC3E51C94FA7436
:1010E3008094805002051C200108AFFBEF600312BF
:1010F3000D46D007D006D005D004D003D002D001CE
:10110300D000D0D0D082D083D0F0D0E0328A358BDB
:1011130036A907E91208ACE0FEA3E0C39DFFEE9CED
:10112300AB07FAE99000C71208D330050B7C007DAA
:10113300091200480D1200AF1208F040037F00228D
:10114300D3EB9536E5351208F440037F0122C3EA59
:101153006480948040037F0222C3E49536FFE495C4
:1011630035FE1208F07F0440027F03227855E6140F
:101173006006047053020C6830003CC2009000F912
:10118300E0049000F8F0120E14D204E54D640260FE
:1011930003120A8DE54D640160031204A7300408AD
:1011A300300205E58730E203120A7C9000D3E07039
:1011B300063002031206899000D8120A194009E486
:1011C300F5F875FB3F120F7122E4FEEEC39406504F
:1011D30042EEFDE54B2DFDE433FC7860E6FBC3ED09
:1011E3009B7480F86C98401AAF067D0E12135FEE65
:1011F30004FCECC39406501BAF04E4FD12135F0C14
:1012030080F0AF06E54B2E2456F8E604FD12135F7B
:101213000E80B843F88022900139E0FD900138E058
:10122300FCC39D5006C3ED9CFE800DED2414FE907F
:101233000138E0FDC3EE9DFEEED3940174809480EB
:1012430040D5C2AC9001381214E92408F8A607204F
:10125300070ED2AC1214E82408F8E6F599D2072257
:10126300D2AC22C0E0C0F0C083C082C0D075D00031
:10127300C000C001C002C003C004C005C006C0074F
:101283003098031214D3309903120003D007D00609
:10129300D005D004D003D002D001D000D0D0D0826A
:1012A300D083D0F0D0E032A90774FFF536F537AF1D
:1012B3004EE4FEE9254EFDE433FCEFC39DEC648070
:1012C300F8748098502175F002EF1208AFE0FCA388
:1012D300E0FDC39537EC95365009900099EEF08CFC
:1012E300368D370F0E80CC2290FC017480F0E49091
:1012F300FC06F090FC05F090FC017481F0A3E0FF84
:10130300E48F35F534F533F532AE34AD33AC321208
:10131300149112148D12148DF532E490FC01F0AC8B
:101323003222900000E004F0E0C3940474809480BF
:101333004029E4F0FF7860E6FEEFC39E501574EA9F
:101343002F1209A5E0600974EA2F1209A5E014F031
:101353000F80E29000D7E0600214F022EF146016D1
:1013630014601914601C14601F1460222405702378
:10137300ED4440F5FC22ED4440F5FD22ED4440F5FB
:10138300FE22ED4440F5FF22ED4440F5F122ED4409
:1013930040F5F2228F33753408D3E534940074801A
:1013A30094804025D287E53330E7047F1780027F9E
:1013B3000D7E001214B9C2877F087E001214B9E5AE
:1013C3003325E0F533153480D0228F32D3E53294C0
:1013D30000748094804027D2877F0C7E001214B95A
:1013E300C2877F287E001214B9D287AF1D121397CC
:1013F300AF1E121397AF54121397153280CE22905B
:10140300801D7404F0E4FF7860E6FEEFC39E501D78
:1014130074562FF8E675F003A424A1F582E434167C
:10142300F58312025874041200360F80DA22E4F5B1
:1014330035AF35C3EF120A12501EE54B2F1209EFD9
:10144300500BE54B25352456F8E6048001E4FDAF47
:101453003512135F053580D943F88022C3EF9DFF12
:10146300EE9CFED3EF9BEA6480F8EE6480985017FD
:10147300C3E49BFDE49AFCC3EF9DEC6480F8EE6447
:10148300809840037F01227F0022F532FCE4FB7A3F
:1014930001F9F81200FB8F358E348D338C3290FCBA
:1014A30002E0FFE5354FFFE534FEE533FDE5328F1E
:1014B300358E348D3322EF1FAA0670011E4A600F4A
:1014C300E4FDEDC394477480948050EA0D80F322C9
:1014D300C2989001221214E92424F582E43401F520
:1014E30083E599F022A3E004F0E075F01484E5F0BD
:1014F300F0E022E53825E025E0229000D8E004F072
:101503007861E66001169000D3E0600214F022EDEA
:1015130090169C93FE74EA2FF582E43400F583EE73
:10152300F022015300015400011F0041000000019B
:101533004A0000000000000101010102020202034F
:10154300030303040404040505050506060606074C
:1015530007070708080808090909090A0A0A0A0BFC
:101563000B0B0B0C0C0C0C0D0D0D0D0E0E0E0E0FAC
:101573000F0F0F101010101111111112121212135C
:10158300131313141414141515151516161616170C
:1015930017171718181818191919191A1A1A1A1BBC
:1015A3001B1B1B1C1C1C1C1D1D1D1D1E1E1E1E1F6C
:1015B3001F1F1F202020202121212122222222231C
:1015C30023232324242424252525252626262627CC
:1015D30027272728282828292929292A2A2A2A2B7C
:1015E3002B2B2B2C2C2C2C2D2D2D2D2E2E2E2E2F2C
:1015F3002F2F2F30303030313131313232323233DC
:10160300333333343434343535353536363636378B
:1016130037373738383838393939393A3A3A3A3B3B
:101623003B3B3B3C3C3C3C3D3D3D3D3E3E3E3E3FEB
:101633003F3F3F000004B000000960000012C000FB
:1016430000258000004B00000096000000E1000030
:1016530001C20001A0001F00D0001F0068001F008E
:1016630034001F001A001F000D001F000A001B009A
:1016730005001B0004003200050032000700500083
:10168300090032000A0032000C0032030B08061472
:10169300251F250102040810200264501E1E01802C
:1016A300190180180180070180060180050180046B
:1016B30001800301800201800101800001801C017F
:0516C300801B01801AEC
:00000001FF
